:020000040800F2
:10500000A01A0020D55000085D8600086D7D0008BC
:105010000000000000000000000000000000000090
:105020000000000000000000000000000D900008DB
:105030000000000000000000518E000809910008E7
:10504000E7500008E7500008E7500008E750000864
:10505000E7500008155B0008E7500008E75000081B
:1050600000000000E7500008515A0008E75000080F
:10507000E75000084D82000800000000E7500008DB
:1050800000000000E75000080000000000000000E1
:10509000E750000800000000E7500008E750000853
:1050A000E7500008E7500008E7500008F1990008B1
:1050B000E7500008E7500008000000000000000072
:1050C0000348854600F060FC00480047C1A700087F
:1050D000A01A00200448804704480047FEE7FEE786
:1050E000FEE7FEE7FEE7FEE7A5910008C1500008D5
:1050F00030B50B46014600202022012409E00D4670
:10510000D5409D4205D31D469540491B25469540F7
:1051100040191546521E002DF1DC30BDF0B51FB40C
:105120000646002082B005464024019100901BE015
:10513000019922460F46304600F04EFB049A059B2B
:10514000801A994110D310461946224600F034FBCC
:10515000361A8F410197224601200021009F00F05E
:105160002BFB38184D4100902046641E0028DFDCE0
:10517000019B00982946324607B0F0BD03460B4319
:105180009B0703D009E008C9121F08C0042AFAD2FD
:1051900003E00B780370401C491C521EF9D2704783
:1051A000D2B201E00270401C491EFBD270470022BF
:1051B000F6E710B513460A4604461946FFF7F0FF16
:1051C000204610BD30B504460020034600E05B1CBD
:1051D000934203D2E05CCD5C401BF8D030BDF8B503
:1051E00002464A40D40F42004B0052085B089A42E4
:1051F00002D20246084611464A0023D0C30D4A0097
:10520000DDB2120EAD1A202D35DA49020126490A07
:10521000F6058A19002C00D0524220214F1B11465E
:10522000B9402A411018C20D9A4221D0002C17D043
:10523000012D08DCDA05801AD20F8019D207DBB203
:1052400000F0F6FAF8BDDA05801A012340001B06CB
:10525000C01880185A428018CA0F1043490007E04E
:105260004908C2071143DA05801A801940088018DE
:1052700000F0D6FAF8BD61000122511A001BF7E7D1
:105280000122D2075140AAE70122D2075040A6E7E7
:1052900070B502464A40D50F40004A00ED0740086D
:1052A0005208002814D0002A12D0C40DD30D410298
:1052B0000120C0055202490A520AE41A09181218BC
:1052C0007D34914201D3641C00E04900002C01DAD6
:1052D000002070BD0023914201D3891A0343400886
:1052E00049000028F7D100290AD0914202D10121BA
:1052F000C90705E0914201D2012101E00121C94322
:10530000E005C018401900F08BFA70BDF0B50746F3
:105310000846584087B0C00F049048000E46590018
:1053200040084908BC1A884105D2384631461E4615
:1053300017460B4602465800400810434CD0300D2B
:10534000039040055900400D490D0590401A029008
:10535000402872DA18030121000B09050843019067
:1053600004980092002805D00199524200208841FB
:1053700000920190029840210A1A0199009800F0C9
:105380001BFA05460C466B4607CB00F036FAC019EF
:105390007141039A0E0D0023D71756401A467A40E2
:1053A000164344D0049A002A2DD0029A012A039A67
:1053B00015DC1205C01A914101263605001C714109
:1053C000D20F059ED2070093019202962A462346E9
:1053D00000F074FA07B0F0BD38463146FAE716051A
:1053E000224A0F46B218C01AB74101210905001C14
:1053F0004F4100187F41114618187941E20F1043C0
:105400006D19644113E0E2076D0815436408C20793
:105410001443039A01261205C01A91413605001C57
:105420007141CE07400830434908C01851412A460F
:10543000234600F036FACDE7FFE70498012240004A
:10544000C117121A00238B4104983146C417381A29
:10545000A141EEE730B40124E407634030BC55E7D6
:1054600030B40124E407614030BC4FE70000E0FFA6
:10547000F0B51FB488B00B990998002448400999E9
:10548000C00F490049080991C0070B9900904900D5
:1054900049080B9109990898A64608431CD00B9916
:1054A0000A98084318D0099801244000420D48008A
:1054B000410D099824050003000B204309900B9827
:1054C0000003000B20430B9050181C494018002289
:1054D00001901446104605E0002001460DB0F0BDD5
:1054E000032801DA034600E003239C46C11A0AAEF2
:1054F0000AE05F0008ADED5B4F00F75B7D430027DE
:10550000AA187C41491C5B1E6145F2DD410004ABD9
:105510005A522104120C0A43240C401C0828DFDBD9
:10552000019802900099704601910090059B049AA1
:105530000799069800F0C2F9D0E700000DFCFFFFC4
:10554000F0B50C465C4085B0E40FE40703944C00D2
:1055500000266408590094464908024602962243F0
:1055600021D062460A431ED06200570D4A000E0346
:105570002303550D012402462C492405781B1B0BDF
:10558000360B401823432643614600901C46501AB0
:10559000B44103D30098401C009002E09218009898
:1055A0005B41002803DA0020014605B0F0BD002071
:1055B000012109050746864611E064461D46141B75
:1055C000B54106D36546521BB341744607430C43AD
:1055D000A646CD0740084908284392185B41054676
:1055E0000D43EAD11046184313D060461946504087
:1055F0007140084306D06046101AB34106D201221A
:10560000002306E000220123DB0702E00122D2434F
:105610005310009874460105381C6141029C039D9B
:105620000019694100F03DF9BFE70000FD030000EB
:10563000C217C10F504010B54018CA079623002169
:1056400000F0F6F810BD10B500229623114600F0C8
:10565000EFF810BD0EB5C217C10F5040CA07401871
:105660000021054B0293019200910A460B4600F07F
:1056700025F903B000BD0000330400000EB5054954
:105680000291002100910A460B46019100F016F9A3
:1056900003B000BD33040000410040020122400A73
:1056A000D205090E80187F2901DA0020704796295B
:1056B00003DC9622511AC8407047963988407047DB
:1056C00070B5CD0F4A0009030123090B1B051943CF
:1056D0000B4BED070024520D9A4201DA002070BDF9
:1056E000074B34339A4203DC9A1A00F075F802E053
:1056F0000449511888402C43F1D0404270BD00004D
:10570000FF030000CDFBFFFF4A0009030123090B43
:105710001B051943094B10B5520D9A4201DA0020BE
:1057200010BD064B34339A4203DC9A1A00F054F849
:1057300010BD03495118884010BD0000FF03000050
:10574000CDFBFFFFC20FD207400040080BD0C10DB8
:105750000723DB01C91840020905400A1143C208AA
:10576000400711437047002001467047CB0FDB070D
:10577000490010B5490802460A4307D00A0D07241C
:105780000903E401090B121B002A01DC002010BDF3
:10579000C900440F0C43C100E018D205801800F086
:1057A0003FF810BD0122D207002800DB101A0029A3
:1057B00000DB511A8142704710B5202A04DB0146F4
:1057C000203A9140002010BD914020239C1A0346AE
:1057D000E3401943904010BD10B5202A04DB084671
:1057E000203AD040002110BD0B46D340D0402024A9
:1057F000A21A91400843194610BD10B5202A06DBB5
:10580000CB170846203A1041C1170B4306E00B4660
:105810001341D0402024A21A91400843194610BDDC
:10582000002904DA401C490001D1400840007047BB
:1058300070B40024050C05D11024000402D1002905
:1058400021D01124050E01D100020834050F01D129
:105850000001241D850F01D18000A41C002801DB5C
:105860004000641C002908D020252E1B0D46F54061
:10587000A14000D001212943084301061B1B000A57
:10588000DB1D02D5002070BC7047DB05181880189E
:105890000029F8DA401C4900F5D170BC40084000EE
:1058A000704710B5002B08DA0024401C61419218A3
:1058B0005B411A4301D14008400010BDF0B51FB450
:1058C00082B005460C0003D0084604F04FF902E010
:1058D00004F04CF920300246009021462846FFF79C
:1058E0006BFF049B059A04460F4618431143084377
:1058F00014D0184610431BD0009840210A1A1846AD
:105900000599FFF769FF05460E46009A0599049828
:10591000FFF752FF084305D0012004E02046394636
:1059200007B0F0BD0020C11705430E432C43374399
:1059300000990E986305401A7905E40A00220C4389
:10594000FD0A0A3002D500200146E9E701051019D9
:1059500069410C9C0D9D00196941FFF7A2FFDFE72B
:1059600010B5002904DB0124E40740428C412146A4
:10597000002B04DB1C460123DB075242A341994262
:1059800000D1904210BD0000064C0125064E05E0F6
:10599000E36807CC2B430C3C98471034B442F7D350
:1059A000FFF792FB48AB000868AB000838B5044627
:1059B000064805490068FFF79BFB604300E0401E76
:1059C00000900028FBD138BD40420F00F8000020B5
:1059D000F8B50446006881688907890F012902D15A
:1059E0000168C90722D18168114A1026114001259A
:1059F00000290ED18168294381600120FFF7D6FF7D
:105A000000F09CFF07460CE000F098FFC01B0A283E
:105A100007D9606D30436065A06D2843A065012003
:105A2000F8BD20680068C043C007EDD10020F8BD74
:105A30001700008010B500231A4603E0845CE318C9
:105A40009BB2521C8A42F9D3D84380B210BD0000E9
:105A500010B5034800F036FD024800F033FD10BDDC
:105A60003C160020F415002030B5446C1C252C4059
:105A70000125A540046C6560046863608368102B91
:105A8000036803D099600068C26030BD9A60006806
:105A9000C16030BD10490120487202205E31487259
:105AA00003203C39487204200E3948720A4B0B49D6
:105AB0005A1C0878587149789971233318715971B3
:105AC000203318775977107551751A461E321075A4
:105AD00051751076517670472C110020E00000209F
:105AE00010B503F069FA202003F004FB012004F054
:105AF000EDFB002003F0FEFA044804F08BFA0448A2
:105B000004F034FD002004F069FD10BDA800002061
:105B10008380000070B505200121000700F002FF1E
:105B200000240D4D002800D02C6002210B4800F00D
:105B3000F9FE002808D10A482C6000880A21484351
:105B40000849088003F066FF012000F023FE0220D0
:105B500000F020FE70BD0000F000002000040050A6
:105B6000CC000020DC0000207047000010B5084980
:105B700000224A6107494B684C1523434B604B6830
:105B8000082423434B60C009C001026010BD00001F
:105B900084160020002002407FB500250C460646F2
:105BA000039500F0C7FDE009029003A90196009556
:105BB000684600F057FD002804D000F08FFD00205B
:105BC00004B070BD00F08AFD0120F9E710B5002394
:105BD00002E0C45CCC545B1C9342FAD310BD0000BD
:105BE00010B5214A00219069C305204804D54169B8
:105BF000022319434161911593699B0505D54369BA
:105C00000124234343616302194393695B0505D56E
:105C10004369082423434361E301194393691B0546
:105C200005D54369042423434361630219439369FF
:105C30009B0405D543691024234343616302194340
:105C400093699B0304D5446920231C434461194391
:105C50009369DB0305D54369402423434361A002D4
:105C60000143916110BD0000002002408416002015
:105C700070B5054600F062FE0646184C0AE0681C46
:105C800008D0002D04D000F059FE801BA84201D995
:105C9000032070BDA069C007F1D1A069800701D5BC
:105CA0000220A061A069C00511D4A06980050ED4AE
:105CB000A06940050BD4A069000508D4A069800440
:105CC00005D4A069800302D4A069C00303D5FFF7FF
:105CD00087FF012070BD002070BD00000020024041
:105CE000F8B51746002605460C4600F023FD09E0EE
:105CF00029460220226800F0FFFC002804D1241D60
:105D00002D1D361DBE42F3D300F0E8FCBE4201D289
:105D10000020F8BD0120F8BD10B50849024600205A
:105D2000054B497905E044001C5B944203D0401CBC
:105D3000C0B28842F7D310BD6E1200204800002088
:105D400010B5094800F0A4FF80B2FFF797FC074A9E
:105D5000074BFFF78DFB0022064BFFF7F1FBFFF728
:105D6000D3FC80B210BD0000B0140020F853E3A5AE
:105D70009B843E4000408F40F8B5414CE0790028BC
:105D800001D0002000E00120E0713D493D48CA7982
:105D90000275097A41753C490A780276497841765C
:105DA0003A48017837481330017005214172962036
:105DB00004F0CCFB4B20C00004F0E2FB3149002290
:105DC00013310C2004F0ACFC00210C2004F0BAFCD0
:105DD000022004F00BFC2E4D00210F2004F030FBBC
:105DE0002842E062F8D0E06A411C3BD0294E2A4F9D
:105DF000400439D58122D20100210F2004F065FC36
:105E00000021102004F01CFB41061E48490E002210
:105E1000633004F04BFB1B4D6335687A052820D1B5
:105E200002221949681DFFF7CDF9002819D1A87A77
:105E3000607113480422691C4030FFF79FF9206C01
:105E400000F02EF860836079294642000B31084645
:105E50007330FFF793F9608B318848433880022014
:105E60002070F8BD02F01EFC0C480188608B0546CE
:105E7000FFF73EF93088414339806D1E6583F8BDD8
:105E8000480000208D110020E0000020BE0000200E
:105E900000D02724C6000020C4000020C800002035
:105EA00010B504460E4800F0F3FE0E49C006C00EC1
:105EB000098805E02246C240D2070FD0401CC0B27C
:105EC0008842F7D3012005E02246C240D20705D020
:105ED000401CC0B28842F7D3491EC8B210BD0000B2
:105EE000B0140020C800002010B5084800F096FA51
:105EF0000A21064800F032FA044800F01DF9800536
:105F000003D5024800F01AF980B210BD54140020E5
:105F1000F8B52F4D00220121284600F008FDFFF7BB
:105F2000E3FFFFF790FB2B4E3146FFF7B1F92A4C08
:105F30000122A0601146284600F0F9FC2749A0681C
:105F4000002588423EDB2078254F002815D025709B
:105F5000FFF7CAFFFFF777FB3146FFF799F9A0601B
:105F6000FFF7F0FB00223B46FFF774FA00221D4BBF
:105F7000FFF77EFAFFF7FAFB6060A068FFF7E2FB2D
:105F800000223B46FFF766FA174A184BFFF770FAF4
:105F900006460F466068FFF7D5FB134A144B524282
:105FA000FFF766FA32463B46FFF7B0F9FFF7DEFB34
:105FB00010496060884201DD616004E0FF21C9058D
:105FC000C84200D365606068FFF766FBC0B2F8BDE9
:105FD0000004005000401B442400002000006040EA
:105FE00000000C4000E064403333333333B33040BF
:105FF000CCCCEC3F0000C842F8B50546044640351D
:10600000287C0026012808D0012028742068816897
:106010008907890F01290ED101E00220F8BD01682E
:10602000C90708D0606D2021084360650126002063
:1060300028743046F8BD616DFF220132914302227F
:1060400011436165C1688907890F0091C16889089A
:106050008900C1602068816892071143816000F067
:106060006DFC07460EE000F069FCC01B0A2809D948
:10607000606D022188431021084360650020287468
:106080000120F8BD206880680028ECDB2068C1682A
:10609000009A1143C160606D80088000401C6065FB
:1060A000C5E70000F8B506460D464036317C0129AB
:1060B0000DD00121317401688A68520709D5416DFC
:1060C000202211434165002030740120F8BD0220D8
:1060D000F8BD174B6A68D80547109A42154C8A6A72
:1060E0002B6812D05B035B0B1A438A622968490351
:1060F00005D5A1680143A1600A20FFF757FC286875
:10610000800312D5A06838430EE05B035B0B9A4313
:106110008A622968490302D5A1688143A160286881
:10612000800302D5A068B843A06000203074F8BD99
:106130000110000000270140406D70470068006CAE
:106140007047000070B5040006D0606D264600253B
:106150004036002802D006E0012070BDA5653574E8
:10616000204600F0D3F8606DC00603D4216888682B
:10617000400705D5606D1021084360653574EBE775
:10618000606DFF22013290430222104360658868EF
:106190008207920F5B48012A02D10A68D2072BD1ED
:1061A000032362689B079A4205D05B429A4202D061
:1061B0005B009A4209D10A69920092080A6121683B
:1061C0000A6963681A430A610CE00A69920092083E
:1061D0000A6181680F22920491438160816862683C
:1061E000114381602168CA6818239A43CA602168F4
:1061F000CA68A3681A43CA608168012252069143A3
:1062000081608168A28E5206114381602068816896
:10621000C90004D4816801221207114381602068FB
:10622000C168394A1140C1602069E168022825D05F
:1062300000200143204620300278037B52035B009C
:106240001A431143226B1143A26992031143E2697D
:10625000D20311432268D3681943D160616A0A46A8
:10626000FF3AC23A05D0A26A11432268D3681943A3
:10627000D16042780121012A02D00BE00420D8E746
:106280000078002823D0606D202210436065A06D47
:106290000843A065E06B012820681FD00169C90789
:1062A00003D0016949084900016120684169C908B2
:1062B000C900416120684169A26B11434161A56534
:1062C000606D80088000401C6065002070BD206803
:1062D000C26801231B041A43C260DBE70269FF2383
:1062E0009B009A43026120680269236CA66C1A43E2
:1062F000636C33431A430261206802690A430261F6
:10630000D3E70000002701401902FEFF10B586B058
:10631000044614216846FEF74AFF0E492068884269
:1063200016D10D48416B421511434163C16A0122E8
:106330001143C162C06A6946104005900220009076
:1063400003200190002002900520000700F02EFAA3
:1063500006B010BD0024014000100240F8B504460C
:106360004069254640350E4608280BD02068C06895
:10637000C00709D0606D20210843606500202874A3
:106380000120F8BD082700E00C2700F0D7FA0090A4
:1063900011E0701C0FD0002E05D000F0CFFA00994C
:1063A000401AB04207D9606D04210843606500209F
:1063B00028740320F8BD206800683842E9D0606D79
:1063C00001214902084360652068C16809058A0FF8
:1063D0000C21002A1BD12022125D002A17D102684D
:1063E000120714D5826853070122002B08DB43688B
:1063F0008B434360606D130298431043606506E071
:10640000606D202318436065A06D1043A065A069EE
:10641000002801D1206801600020F8BD70B5044655
:10642000216800208968490721D425464035297C08
:1064300001291CD001212974E169012904D02046D9
:10644000FFF7C6FA002811D1616D0A4A1140FF22F8
:106450000132114361650021A165297422681C2164
:10646000116021688A6804231A438A6070BD022083
:1064700070BD0000FEF1FFFF70B500240146203121
:106480004A79022A03D00421C163012418E002687A
:1064900013680E25AB431360026813685B085B004A
:1064A0001360436C1C221340012215469D40036C6F
:1064B0005D604A7100220A71816B002900D0884713
:1064C000204670BDF0B4016C0D6801680C68466C24
:1064D0001C2304221E401746B7402F420ED06707E8
:1064E0000CD50C68A40602D40C6894430C60416C73
:1064F00019408A40016C4A60016B1AE00227B740DC
:1065000002462F402032002F17D0A70715D50C6860
:10651000A40605D40C680A25AC430C600121517116
:10652000446C02211C40036CA14059600021117190
:10653000C16A002918D0F0BC08470827B7402F428D
:1065400012D0240710D50C680E25AC430C60446CA7
:1065500001211C400B46A340046C6360C163517170
:1065600000211171416BE4E7F0BC704770B5040085
:106570003CD01F48256814212818FEF7B9FD80007B
:1065800060641C482064022120462030024641718C
:1065900029681948E3680140A068666918432369BF
:1065A00033431843A3691843E3691843236A184324
:1065B000084328600121A0688903884210D00D4853
:1065C0008030836A656C1C210D400F26AE40B343BA
:1065D0008362656C63680D40816AAB400B438362E4
:1065E0000020E06301215171107170BD012070BD68
:1065F000F8FFFDBF000002400F80FFFFF8B5044622
:106600008C46203001790025012909D00126067128
:1066100041790027012905D0077102252846F8BDD8
:106620000220F8BD02214171E76320680168490832
:106630004900016061462046FFF716FA206B0028EA
:106640002068016801D00E2205E004229143016018
:10665000206801680A221143016020680168314303
:106660000160DBE7F8B51A4E0546307C0F4601287D
:1066700007D0012030741748FFF7FAFA010002D062
:1066800021E00220F8BD0020C04338606C6814E0AF
:106690002046FFF76BFA0F48FFF7EAFA01460E486B
:1066A000426808239A434260426843159A43426015
:1066B000002901D03C6006E08034A8686A68C00107
:1066C0008018A042E4D8002030740846F8BD0000CD
:1066D0008416002050C30000002002400548416895
:1066E00002221143416041680122114341600020B0
:1066F0007047000000200240F8B50C4C1646207C84
:106700000F46012808D0012020740948FFF7B0FA8D
:106710000025002802D006E00220F8BD65613E6039
:106720000348FFF7A5FA2574F8BD00008416002081
:1067300050C3000011484168C9070BD0EFF3108126
:1067400072B60F4AC2600F4AC26081F31088416876
:10675000C9070ED1416889070DD5EFF3108172B6D4
:10676000094A0261094A026181F310884068800782
:1067700001D5012070470020704700000020024032
:10678000EFCDAB8905040302BFAE9D8C1615141323
:106790007047000010B504494A69024202D04861BE
:1067A000FFF7F6FF10BD000000040140F8B500231C
:1067B0000124A2E027469F403A4070D04D68022D48
:1067C00001D0122D14D1DD08AD002D1800952D6AD1
:1067D0005E07AC46F50E0F26AE46AE406546B543A5
:1067E000AC460E697546AE4065462E43009D2E624E
:1067F0004D68012D05D0022D03D0112D01D0122D91
:1068000016D185680326AC465D00AE46AE406546AF
:10681000B543AC46CE687546AE4065462E438660AD
:1068200046680D79BE43ED06ED0F9D40354345604A
:1068300006685F000325BD40AE46AE430D79B44601
:10684000AE07B60FBE4065462E430660C668754665
:10685000AE438D68BD403543C5604D68ED004BD5F6
:10686000294D6E6B26436E639E08284DB600751940
:10687000AC46AD689E07360F0F27B740BD430527CE
:106880003F07B84201D1002715E0214FB84201D19E
:10689000012710E01F4FB84202D102270BE02BE086
:1068A0001D4FB84201D1032705E01C4FB84201D16A
:1068B000052700E00627B7402F436546AF60184D17
:1068C0002E684F689643FF0300D516432E606E680E
:1068D0004F689643BF0300D516436E60AE684F689D
:1068E0009643FF0200D51643AE60EE684F689643AC
:1068F000BF0200D51643EE605B1C0A681546DD40FA
:1069000000D057E7F8BD0000001002400000014031
:106910000004005000080050000C0050001C005003
:10692000000401400069084000D001207047002A9F
:1069300001D08161704781627047000001480068A2
:1069400070470000F400002002480168491C016003
:1069500070470000F400002010B5084800240168CA
:10696000402211430160204600F00AF8002801D0BF
:10697000012401E000F0B8F9204610BD00200240DB
:1069800070B5054609487D210024C9000068FEF75E
:10699000AFFB00F04DFE002801D0012404E00022EE
:1069A0002946501E00F0C0F9204670BDF8000020B6
:1069B00070477047F8B5304C01276078401C607014
:1069C000E770E08B401CE083208902F05DFB2B4DDB
:1069D000E888FEF738FE2A49FEF75AFC294E009057
:1069E0003168FEF7FCFB3060A16AF805814203DBE9
:1069F0000098FEF749FCA06202212348FFF792FFAE
:106A0000002809D00020E0621E482049066820487E
:106A10008E4212DD077012E0E888FEF714FE184976
:106A2000FEF736FCE16AFEF7DAFB1A49E0628842BB
:106A3000EADB1A491848C860E6E700210170688F50
:106A4000401EFEF7F5FD3146FEF7ACFE06D8207974
:106A5000002803D01248C1793943C171688FFEF70D
:106A6000F2FD08490968FEF79DFE04D2207900284E
:106A700001D003F03DFFF8BDBC0000202C0D00202C
:106A800000007A44F0000020000400500000404064
:106A90004E0000200000A0400400FA0500ED00E0D8
:106AA000A0110020704770B505000DD002202C46C3
:106AB0002034A073284601F0D1FB284600F0BEF830
:106AC0000020A073607370BD012070BD70477047D7
:106AD00010B5044600680168C943C90708D1816838
:106AE000C943C90704D1012141602046FFF762FF75
:106AF00020680168C943890708D48168C9438907A8
:106B000004D4022141602046FFF752FF206801684B
:106B1000C943490708D48168C943490704D40421FB
:106B20004160204600F0DEF820680168C94309078B
:106B300008D48168C943090704D40821416020466C
:106B4000FFF7B0FF20680168C943C90608D481680F
:106B5000C943C90604D4102141602046FFF729FF2C
:106B600020680168C943890608D48168C943890639
:106B700004D4202141602046FFF7A9FF2068016866
:106B8000C943490608D48168C943490604D4402151
:106B900041602046FFF79AFF10BD0000F8B50400E1
:106BA00005D025462035A87B002802D006E001202C
:106BB000F8BD00206873204600F052F80220A87348
:106BC0002068C26884466368012B04D00120A16A52
:106BD000C005814201D11E2082431548616981426E
:106BE00001D0144802401448A668024018463043B9
:106BF000676A266A3E433043A66A30431043012B3E
:106C000003D00122D205964203D12369E2681A43D8
:106C10001043074A914205D0A2691143E269024339
:106C2000084610436146C8600120A8730020F8BDE3
:106C3000FFFF00003F1FFFFFF8F119FF10B50068CC
:106C40000549884207D10548816B4900490881639D
:106C50000D2000F055F810BD007C004000100240EF
:106C600010B50068084988420CD10848816BC204FD
:106C700011438163002201210D2000F055F80D2001
:106C800000F048F810BD0000007C004000100240F9
:106C90000068C0697047000070B5022403462033C5
:106CA0009C730F4C2568E604354325600468E5684D
:106CB000B6123543E5600568AE6801242643AE6030
:106CC00005682E6926432E610568A96101684A613D
:106CD000006801690422114301619C73002070BDAA
:106CE00000040140704700000448416B0122114339
:106CF0004163816B020411438163704700100240BD
:106D0000C106C90E01208840014908607047000093
:106D100080E100E0C106C90E0120884001490860F9
:106D20007047000000E100E010B501F099FC10BDD3
:106D300002494A6882434A60704700000070004080
:106D400002480168821511430160704700700040DD
:106D500002494A6802434A607047000000700040E0
:106D600005480168022211430160044801690422B8
:106D70001143016130BF70470070004000ED00E03A
:106D80000A4B1A689208920002431A600848036985
:106D9000042213430361012906D040BF20BF20BF56
:106DA000016991430161704730BFF9E7007000400D
:106DB00000ED00E0F8B504460078544D800672D529
:106DC000524E0027403EB06BC00004D4B06BA90502
:106DD0000843B06301274E480168C90511D4016812
:106DE000821511430160FFF7A9FD009005E0FFF750
:106DF000A5FD0099401A642837D845480068C005A9
:106E0000F5D532680321090560680A4001409142C6
:106E100008D08103890F032904D13168890301D582
:106E20000120F8BD2A69032109040A4022D0084044
:106E300090421FD0207880061CD528692A69884393
:106E40000121C9040A432A612A698A432A61286107
:106E5000C0050FD5FFF772FD009008E0FFF76EFD4B
:106E60000099411A2B48814201D90320F8BD2869B5
:106E70008005F3D561688803800F032805D1326847
:106E80000005824301400A43326028690322616899
:106E90001204114008432861002F04D0B16B012077
:106EA00000078143B1632078C00705D0E868A16876
:106EB000800880000843E8602078800705D5E868EE
:106EC0000C218843E1680843E8602078400706D534
:106ED000E86803218902884321690843E860207833
:106EE000000706D5E8680321090388436169084360
:106EF000E8602078000606D5E86803218904884305
:106F0000A1690843E8600020F8BD0000401002407D
:106F10000070004088130000F8B50E4605007DD0D3
:106F200053480068C007C00FB0420AD250480168F9
:106F300049084900314301600068C007C00FB042F2
:106F400071D128784B4C800705D5E068F021884343
:106F5000A9680843E0602878C00752D06868022812
:106F600017D0032818D02168012818D089050029D6
:106F700059DAE168890889000143E160FFF7DEFC26
:106F800069680746022912D003291CD0012926D09E
:106F900033E021688903EAE721688901E7E74907C7
:106FA000E5E7FFF7CBFCC11B3348814223D8E068FB
:106FB0000007800F0228F4D123E0FFF7BFFCC11BBC
:106FC0002D48814217D8E0680007800F0328F4D1CC
:106FD00017E0FFF7B3FCC11B274881420BD8E068DC
:106FE0000007800F0128F4D10BE0FFF7A7FCC11BBD
:106FF0002148814201D90320F8BDE0680007800FD5
:10700000F3D11B480168C907C90FB1420DD9016806
:107010004908490031430160006800E003E0C0070F
:10702000C00FB04201D00120F8BD2878400706D536
:10703000E068072109028843E9680843E06028788E
:10704000000707D5E0680721C90288432969C900FC
:107050000843E06000F036F8E168084A0906090FC5
:10706000515CC840064908600020FFF789FCF8BD64
:1070700000200240001002408813000026AB0008E8
:10708000F8000020044805490068C968044A490519
:10709000490F515CC8407047F800002000100240C2
:1070A0003FAB0008044805490068C968044A8904E0
:1070B000490F515CC8407047F800002000100240A2
:1070C0003FAB000810B5184AD1680C2008400428CE
:1070D0000BD0082810D00C2810D050680004410FA5
:1070E0000120C003491C884010BD1068C00601D5AE
:1070F0000E4810BD0E4810BD0E4810BD88020E4B44
:10710000000F185C0902D368890F491CDB0301D505
:10711000084A05E01268D20601D5044A00E0044A94
:107120005043FDF7E5FF10BD0010024000093D008F
:107130000024F40000127A0036AB0008FEB505000A
:107140007ED0FE4CE7680C20E66807400120000472
:1071500006402878C00747D0082F05D00C2F0AD149
:1071600001200004864206D1206880033CD568686F
:107170000028E5D038E0012069680004814203D18D
:1071800021680143216011E0052301221B049204C0
:107190009942216802D111432160F1E781432160C6
:1071A00021680140009120689043206068680028B1
:1071B0000DD0FFF7C3FB009005E0FFF7BFFB009980
:1071C000401A64287AD820688003F6D50CE0FFF7CF
:1071D000B5FB009005E0FFF7B1FB0099401A642869
:1071E000F0D820688003F6D42878800755D5092385
:1071F000E868042F0DD00C2F01D1002E09D00028F3
:107200003BD02168994301432160FFF797FB064675
:1072100027E02168490701D5002891D061681F2225
:10722000120291432A691202114361602168994355
:1072300001432160FFF746FFE16809060A0F00E0FD
:1072400079E1BF49895CC840BE4908600020FFF76A
:1072500097FB002872D120E0FFF770FB801B02280B
:10726000B0D820684007F7D560681F21090288431D
:1072700029690902084360600FE020684008400067
:107280002060FFF75BFB064604E0FFF757FB801B1F
:10729000022897D820684007F7D42878C0065FD521
:1072A000002F0CD0A869002849D02068FF210131A7
:1072B00008432060FFF742FB06462DE0C0E020684F
:1072C000800502D5A8690028A7D060680721490376
:1072D0008843296A084360606068297F0002000AC9
:1072E000090608436060286A410B0120C003491C5D
:1072F0008840E16809060A0F9149895CC8409149B4
:1073000008600020FFF73CFB002817D128E0FFF7BA
:1073100015FB801B0228A3D820688005F7D560687C
:10732000072149038843296A084360606068297F10
:107330000002000A09060843606011E0E1E02168EC
:10734000FF20013081432160FFF7F8FA064604E090
:10735000FFF7F4FA801B022872D820688005F7D462
:107360002878794E000724D568690028306910D044
:10737000012108433061FFF7E1FA009005E0FFF7D3
:10738000DDFA0099401A02285AD830698007F6D5EC
:107390000FE0400840003061FFF7D0FA009005E0B0
:1073A000FFF7CCFA0099401A022849D830698007C3
:1073B000F6D42878400765D500200290A06BC00065
:1073C00006D4A06B012109070843A06301200290A5
:1073D0005E480168C90511D4016882151143016036
:1073E000FFF7ACFA009005E0FFF7A8FA0099401A01
:1073F000642825D855480068C005F5D5FF20AA683F
:107400000130824203D131690143316111E0012130
:107410008902002A07D005231B029A4203D1326950
:107420000A433261EFE7326982433261306988434F
:107430003061A86800280FD0FFF780FA009007E0BD
:107440005EE0FFF77BFA0099411A4148814257D824
:1074500030698005F5D50DE0FFF770FA009006E081
:10746000FFF76CFA0099411A3948814248D83069CF
:107470008005F5D40298002804D0A06B01210907EB
:107480008843A063686A002864D00C2F3ED0012690
:1074900036060228206805D0B0432060FFF74EFA78
:1074A00005462FE0B0432060FFF748FA074604E0A6
:1074B000FFF744FAC01B022822D820688001F7D4C5
:1074C000E96AA86AE2680843296BFD231B049A4312
:1074D00011430843E060206830432060FFF72EFA34
:1074E000054604E0FFF72AFA401B022808D8206866
:1074F0008001F7D52EE0FFF721FA401B022801D9C1
:107500000320FEBD20688001F5D423E00128F8D0D7
:10751000E06801210904AA6A014091420BD10F21C0
:107520008904EA6A0140914205D103218905084096
:10753000296B88420ED00120FEBD000000100240E1
:1075400026AB0008F8000020401002400070004008
:10755000881300000020EFE770B5040007D0002674
:1075600025464035A662687C002802D005E001204F
:1075700070BD2E74204600F02FF802206874206839
:107580000168402291430160A16860682269084354
:10759000E16811430843616901220843A16952026D
:1075A00011400843E1690843216A0843A16A08437E
:1075B00021680860A0690421000C0840616A084342
:1075C000216848602068C16992009143C161666585
:1075D00001206874002070BD10B586B004461421E7
:1075E0006846FDF7E4FD10492068884219D10F482C
:1075F000416B821411434163C16A01221143C1628C
:10760000C06A002110400590E02000900220019007
:107610000320039002910491052069460007FFF7BB
:10762000C5F806B010BD0000003001400010024057
:10763000094910B5401E884201D9012010BD074CF0
:1076400060610321081F01F00BF80020A0610720F2
:107650002061002010BD0000FFFFFF0000E000E0FF
:10766000F0B502462032137E012B15D00127177684
:107670000223537605686C68AB687026B4430E68C5
:10768000496826438024A34319436E6000688160E3
:10769000577600201076F0BD0220F0BD70B50400D2
:1076A00005D025462035687E002802D006E001205E
:1076B00070BD00202876204600F00AF80220687687
:1076C000211D206801F09AFD01206876002070BD20
:1076D000006801218907884204D10348816B012297
:1076E000114381637047000000100240F8B5054661
:1076F00004462035287E012817D001262E76022048
:107700006876226890687727FF23B8431B02984366
:1077100090600A68502A31D00EDC202A4BD006DC5B
:10772000002A48D0102A3AD145E00220F8BD302A7C
:1077300041D0402A33D136E0602A27D0702A12D0B7
:1077400001200003121A2AD0824228D1CB684A684D
:107750008968206801F08BFD20688168012292030E
:10776000114381601BE0CB684A688968206801F09A
:107770007EFD216888683843886010E0CA684968DF
:10778000206801F0EEFD5021206806E0CA684968D3
:10779000206801F0F7FD6021206801F073FD6E762E
:1077A00000202876F8BDCA684968206801F0D9FD34
:1077B00040212068F1E711462068EEE710B586B059
:1077C000044614216846FDF7F2FC01212068890770
:1077D000884212D10A49CA6A02200243CA62C96AAF
:1077E0000190014005914102009100210291039115
:1077F000049069460348FEF7D9FF06B010BD0000AB
:107800000010024000040050F8B506460446203639
:10781000307E0D4601280DD0012030760220707692
:107820000427002A08D0042A16D0082A2AD00C2AB5
:107830004DD137E00220F8BD206801F02BFD206813
:10784000816908221143816120688169B94381619E
:1078500020688169EA6812E0206801F033FD206841
:1078600082690121C9020A4382612068816901227B
:1078700092029143816120688169EA681202114392
:10788000816124E0206801F036FD2068C26908218A
:107890000A43C2612068C169B943C1612068C169F6
:1078A000EA6812E0206801F041FD2068C169012208
:1078B000D2021143C1612068C269012189028A4351
:1078C000C2612068C169EA6812021143C1610120E6
:1078D000707600203076F8BD70B5040005D02546DE
:1078E0002035687E002802D006E0012070BD00200F
:1078F0002876204600F00AF802206876211D2068CC
:1079000001F07CFC01206876002070BD704710B546
:1079100004460068012201F09DFC20688168490747
:10792000490F062903D0016801221143016000209C
:1079300010BD000010B504460068002201F08AFC6A
:107940002068016A054A114203D1016849084900CB
:107950000160012020346076002010BD111100006C
:1079600070477047F8B502680446D069116893689B
:1079700005072D0F5BD0DD07ED0FFF2621360E40EA
:107980002E4367D0C60706D0CE0504D50126166261
:10799000E26F3243E267870702220426002F06DAED
:1079A000DF0704D027683A62E76F3743E767470786
:1079B00006D5DB0704D023681E62E36F1343E36739
:1079C000020709D520220A402A4305D0236808224D
:1079D0001A62E36F1343E367E26F002A2FD0800639
:1079E00006D5880604D5216E002901D02046884797
:1079F000E06F21688968490601D4000724D5204634
:107A000001F066FE20688168490619D58168402228
:107A100091438160E06E002812D020498163E06EBE
:107A2000FEF72AFD00280AD0E06E816B06E085068D
:107A300010D58D060ED5216E1CE020468847F8BD76
:107A40002046FFF78EFFF8BD2046FFF78AFF002093
:107A5000E067F8BDC50208D55B0206D50120000528
:107A600010622046FFF77CFFF8BD030605D50B0624
:107A700003D5616E0029E0D1F8BD4006FCD548066B
:107A8000FAD51368204640218B431360202161679B
:107A90000021616600F069F9F8BD00002D9600082C
:107AA00010B5040003D0606F002802D007E0012069
:107AB00010BD002170200155204600F027F8242039
:107AC000606720680168490849000160204601F0AC
:107AD00049FE0128ECD0606A002802D0204601F05F
:107AE00087FC206841680922D202914341602068E6
:107AF00081682A2291438160206801680122114334
:107B00000160204601F0DAFC10BD0000F0B587B03E
:107B1000064614216846FDF74AFB2C493068884226
:107B200051D12B48416B0122920311434163C16A39
:107B300001221143C162C06A002510400590032054
:107B4000400200900220032701A9A1C10420049053
:107B5000052069460007FEF729FE1F4C1D48A56059
:107B6000E56081C48027E560A76020202561606111
:107B70000002A0611848083CFEF7F8FC002801D07C
:107B8000FDF7F2FFF466A662144C12482146143841
:107B900020600320606010200831A1C16561A561EB
:107BA000E56120462562FEF7E1FC002801D0FDF7E3
:107BB000DBFFB466002201211B20A662FFF7B4F8A8
:107BC0001B20FFF7A7F807B0F0BD00000038014008
:107BD0000010024030000240F41500203C16002046
:107BE000F8B50446806F20284DD100290BD0002A1B
:107BF00009D00123A0681B03984206D12069002800
:107C000003D1C80701D00120F8BD25466035287C86
:107C1000012838D0012028745820616502530026BD
:107C2000E6672220A067E06E002819D01749C162DC
:107C3000E16E17480863E16E16484863E06E13462C
:107C40008663676D21683A462431E06EFEF7D6FC04
:107C5000002805D01020E0672E7420206067D2E74E
:107C60002E7420680168FF220132114301602068F0
:107C7000816801221143816020688168402211439C
:107C800081600020F8BD0220F8BD00008996000840
:107C9000C79600084196000870477047FFB5044634
:107CA000406F83B017460D4620285CD1002D0AD0C6
:107CB000002F08D0A168C001814207D120690028A7
:107CC00004D1E80702D0012007B0F0BD20466030A3
:107CD0000290007C012846D0029801210174002006
:107CE000E06721206067FEF729FE264640360190B6
:107CF000378277820120A1680003814202D1206986
:107D0000002802D02F46002511E000270FE00022B6
:107D10008021204601F03AFE002815D1002F15D011
:107D20002168387888627F1C708A401E7082708A51
:107D3000019B002806980090E9D1002240212046AE
:107D400001F024FE002808D00320BDE72888216820
:107D5000C005C00D8862AD1CE6E72020606702996F
:107D600000200874B0E70220AEE7704701490248DE
:107D7000C160FDE70400FA0500ED00E070B586B0D3
:107D800014216846FDF713FA0F480124418B00299E
:107D900000D14483408B012805D0022801D100F096
:107DA000E7FB06B070BD0122084E95022946304619
:107DB000FEF7BDFD002102910391009501946946F3
:107DC0003046FEF7F3FCECE7BC0000200004005056
:107DD00010B505242407002204212046FEF7A7FD44
:107DE000002208212046FEF7A2FD0A2002F0CBF86F
:107DF000012204212046FEF79AFD0A2002F0C3F872
:107E0000002204212046FEF792FD10BD10B5052486
:107E10002407002204212046FEF789FD01220821C3
:107E20002046FEF784FD0A2002F0ADF8012204216D
:107E30002046FEF77CFD0A2002F0A5F8002204216E
:107E40002046FEF774FD10BDF8B500240526074650
:107E500025463607002204213046FEF768FD0A2039
:107E600002F091F8012204213046FEF760FD600621
:107E7000040E08213046FEF755FD002801D0641C91
:107E8000E4B2052002F07FF86D1CEDB2082DE1D3BD
:107E9000002F03D0FFF79CFF2046F8BDFFF7B6FF89
:107EA000FAE770B50526054636070022042130465C
:107EB000FEF73DFD0024E80901D0012200E0002288
:107EC00008213046FEF733FD6806050E0A2002F051
:107ED0005AF8012204213046FEF729FD0A2002F05B
:107EE00052F8002204213046FEF721FD0A2002F05C
:107EF0004AF8641CE4B2082CDDD370BD10B505242B
:107F00002407012208212046FEF711FD0122042149
:107F10002046FEF70CFD002208212046FEF707FD53
:107F20000A2002F030F8002204212046FEF7FFFC70
:107F300010BD10B505242407002204212046FEF7B9
:107F4000F6FC002208212046FEF7F1FC0A2002F090
:107F50001AF8012204212046FEF7E9FC012208213B
:107F60002046FEF7E4FC0A2002F00DF810BD70B5C3
:107F700005252D070024012208212846FEF7D7FCFD
:107F8000062002F000F8012204212846FEF7CFFC6B
:107F9000062001F0F8FF07E0641CE4B2FA2C03D9D4
:107FA000FFF7C7FF012070BD08212846FEF7BAFC85
:107FB0000028F1D1002204212846FEF7B8FC002059
:107FC00070BD0000F8B501F0A9FA01F0E3FA5448D9
:107FD0000068C069534E544F800700D5FE60FDF71E
:107FE000AFFE5249524D898F524C002929D0524937
:107FF0000A7801218902002A05D0012A0ED0022A1E
:1080000010D0032A1DD1608B01282AD0022818D154
:10801000434808213C38FFF78DFC12E0FF22F5327F
:108020009042F0D2608B012819D0022804D008E0D9
:108030002846FEF77CFC04E0394808213C38FFF76D
:1080400066FC0121C9023A48FEF76CFC00250028B5
:1080500029D03A480560A079002804D007E0002222
:10806000E6E70122E4E70120A07101F0D3FC2078CB
:10807000632806D9002208212D48FEF758FC01226A
:1080800005E0012208212A48FEF751FC00220121C7
:108090000520C9030007FEF74AFC244C4034A08C9D
:1080A000012803D01CE0A5710022EBE724486946B3
:1080B000088072B680212348FDF76EFD002804D0A9
:1080C000022269461F48FDF70BFE62B61EA001F0B2
:1080D0003DFDA58402F0A8FC642001F04DFFFE6088
:1080E000608C012808D111486584058002F09CFC51
:1080F000642001F041FFFE60208C012806D1258418
:1081000002F092FC642001F037FFFE600748124A3B
:108110000188914202D1C088002800D1FE60F8BDDC
:10812000741500200400FA0500ED00E02C0D00207D
:1081300000040050BC0000205A000020F000002085
:10814000AAAA0000384A0008BDF8C8EBC9FDBCB6B1
:10815000C4A3CABD0D0A0000AA55000008B5372106
:10816000202000F06EF80321212000F06AF8402161
:10817000222000F066F80821232000F062F8AA21EE
:10818000302000F05EF80A4802210187322000F01A
:1081900058F80121332000F054F85F21202000F02E
:1081A00050F8684600F006F80A2001F0ECFE08BD21
:1081B0002C0D002010B501460F2000F021F80028FA
:1081C00000D0012010BD10B50446FFF797FE322005
:1081D000FFF767FEFFF7CBFEE0B2FFF762FEFFF7A7
:1081E000C6FEFFF78BFE3320FFF75BFEFFF7BFFEF7
:1081F0000020FFF729FE0446FFF79BFE204610BD36
:1082000010B50C46FFF7DFFF2070012010BD70B5E0
:108210000D460446FFF772FE3220FFF742FEFFF7DD
:10822000A6FEE0B2FFF73DFEFFF7A1FE2846FFF7EE
:1082300038FEFFF79CFEFFF77CFE0A2001F0A3FE4C
:1082400070BD10B5FFF7E3FF012010BD10B5024867
:10825000FEF73EFC10BD0000B0140020FEB5044641
:10826000002572B60068394A831804D13849CD68B0
:10827000032189040D4081680191C1680091416921
:108280008669002B08D132484038836AC7043B43D3
:108290008362836ABB4383620846304348D02B48DD
:1082A0002368C34205D12A48C3680322920493433A
:1082B000C360002917D02068026901231A430261B4
:1082C00020684161FEF73AFB0746FEF737FB21685D
:1082D000C01B0968090703D47D21C9008842F4D96D
:1082E000216808204860002E17D02068016901220B
:1082F0001143016120688661FEF720FB7D27064659
:10830000FF00FEF71BFB2168801B0968C90601D42A
:10831000B842F6D92168102048600C482168C14253
:1083200006D10B48C1680322920491432943C160DE
:108330002068016949084900016121680198886045
:1083400021680098C86062B6FEBD00000084FFBFCF
:10835000401002401CB5002116480091144A0191BA
:108360000260C163120542608160072282630122BC
:1083700002610246C16020321170FF235170C23386
:10838000436281621173016381610422416342612E
:10839000C161FDF7D7FE084800908013019069463F
:1083A0000448FDF77FFE00210248FDF725FE1CBDB5
:1083B00000240140541400200200000408B50848BD
:1083C000016B012211430163006B012110400090F9
:1083D00000220A20FEF7A8FC0A20FEF79BFC08BD3D
:1083E00000100240F0B587B014216846FCF7DFFEAC
:1083F0004748C26A04210A43C262C26A0A4005921F
:10840000C16A80263143C162C16A31400591C16AA7
:1084100001242143C162C16A21400591C16A02253C
:108420002943C162C06A22462840059005201C21CC
:108430000007FEF77CFA012236493748FEF777FA43
:10844000002236493448FEF772FA912105200022B5
:1084500009020007FEF76BFA31480190002705205A
:108460006946029700940007FEF7A0F90C200090DF
:108470001120019003200390052002976946000710
:10848000FEF794F910206A46039591C205206946CB
:108490000007FEF78BF911200190029769460397B8
:1084A00000941D48FEF782F91E4801906946009528
:1084B00002941948FEF77AF9E002009069460197A4
:1084C00002951548FEF772F91748694691C1694649
:1084D00011480397FEF76AF991200002694691C19D
:1084E0000520694600070397FEF760F969460A48C8
:1084F000019700960294FEF759F900220121052008
:10850000FEF712FC0520FEF705FC07B0F0BD0000E9
:10851000001002400102000000040050083000007A
:1085200000001110000021100832000010B50F4C9F
:108530000D482060FF20053060600020A060E060F2
:1085400020616061E0610121206249026062A161F5
:10855000A0620720E0622046FEF7FEFF2068016867
:1085600040221143016010BD00300140E0140020A2
:1085700010B58AB0002404940594069407940894D6
:1085800001211848099400940194029489070394E6
:108590000160092184604160046113494461C16044
:1085A000FFF77CF801200003049004A90D48FFF7B1
:1085B0009DF80C48FFF790F9089408A90948099418
:1085C000FFF74EF8602000900848019002940822BE
:1085D000694603940348FFF717F90248FFF7EEF8DE
:1085E0000AB010BD381500209304000057020000A7
:1085F00000B585B014216846FCF7D9FD1648154929
:108600000160E1214902416000218160C160016196
:1086100081610C22C161426101623021416201210C
:10862000090381634900C163FFF73AFA0120800220
:10863000009002200190012002900320039004206A
:108640000490052069460007FEF7B0F801F0DCF958
:1086500005B000BD003801407415002070470000CF
:108660008307FF22DB0E9A408907090E99400028F4
:108670000BDA0007000F0838830808489B00181819
:10868000C36993430B43C3617047830804489B004D
:108690001B181868904308431860704700ED00E00D
:1086A00000E400E0BFF34F8F04490348C860BFF304
:1086B0004F8F00BFFDE700000400FA0500ED00E069
:1086C000F0B58FB0962001F041FF4B20C00001F0C3
:1086D00057FFFF4C00256570A07B0C2801D30B20B1
:1086E000A0730122052051020007FEF720F9A07BAC
:1086F00060736071F748A570F74E00783070F748E6
:10870000022100783071F648FEF70CF9002862D09B
:108710000020A179F04E49000843F071A06AF07082
:10872000401CA06260793146B0724200CE310846EA
:10873000C338FCF723FD06207072304613380290D0
:10874000217F0175617F41756079002240003146CB
:108750000D3001F0E5FF6079002140000D3001F09F
:10876000F1FF022001F042FFF5712574A57201208E
:108770002073E572DB48FEF78BFA20840646A5706D
:108780006079FCF77BFFD84AD84BFCF771FE01F00B
:108790008FFB0022D64BFCF7B9FDFCF7B5FF0006B6
:1087A000C10C881980B20121C9036084884201D3B9
:1087B000401A6084CF486063E078401CE070C9488C
:1087C000FEF766FAE083CC480C90C3484E300B901D
:1087D0001630019027E201209BE7C248FEF758FAC5
:1087E000E083C64EC64F21E0A07A002813D001F0E6
:1087F0006EFE039988420ED9069988420BD201F089
:108800003DFD2573099801F09AFE012001F0EEFE6E
:108810002072A57211E0B348FEF73AFA80B2E08305
:10882000618C884202D3C919884206D300210F20E7
:1088300001F006FE3042E062D6D0E06A411C1FD053
:1088400040047DD58122D20100210F2001F03DFF9F
:108850000021102001F0F4FD41069F48490E00223E
:1088600050300A9101F022FE002001F089FE002024
:1088700001F03BFE984E5036707A0728AAD101E0ED
:10888000FFF710FF02229F49701DFCF79BFC002898
:10889000A0D19148503001788E480078814299D11A
:1088A00000273E460DA801F018FE04200DAA390E3F
:1088B00036020E433902175C0F43401EF7D5A764FA
:1088C000E66400273E46104601F0F9FD04200DA99C
:1088D0003A0E360216433A020F5C1743401EF7D594
:1088E00027656665A1786A46491CA1707A494D31B1
:1088F0000E7916774F7969464F77607B002809D14A
:10890000012275482271898BCE30018062710298F4
:108910000675477570486946CE300088898B059189
:1089200088427DD10B987849008A08806A4826469B
:108930004C30808A20836B48FEF7AAF9F08300E070
:1089400066E1308B7149FF30C33080B2308388429A
:108950000CD9494240186C49308308886B4A401C46
:1089600080B20B320880904200D30D80684903200A
:1089700008700B98564A81891186C089644B5086CD
:10898000903B326B1A601A46B03AD37C1F073F0FF8
:10899000032F00D0B7741A09F274F57001274C4AFE
:1089A000B7729186D0867079FF219131484357493B
:1089B000326D593940180104C817736D8918584130
:1089C0000206080A104353490990401803901921E0
:1089D00009988902401806900998B843010E0002D0
:1089E000F165B0653C48F36C0A30B26C01F0D0FE22
:1089F0003948736D1630326D01F0CAFE3648F36D9A
:108A00001230B26D01F0C4FE334808214172314981
:108A100000220978017070792F4980001C3000E035
:108A20009EE001F07DFE7079002180001C3001F095
:108A300089FE29492648F772042251314030FCF75B
:108A40009DFB3148318B07887D20C000784340185A
:108A5000B0630D9030480078F0730090264840389D
:108A6000C088FCF7F0FD05903846FCF7ECFD059951
:108A7000FCF70EFC7F21C905FCF7B1FBFCF70CFEEF
:108A800081B2254801800098401E814201D1012019
:108A9000F072B7841420305EFCF7DCFD079108907B
:108AA000F08BFCF7EBFD1D4A1D4BFCF7E1FC009140
:108AB0000A900D98FCF7CEFD009B0A9AFCF7CAFCC1
:108AC000079B089AFCF722FCFCF7FAFDF06329E00B
:108AD00048000020BE000020A0110020BC000020A3
:108AE00000040050B0140020666666666666E63FC5
:108AF00000000840A08601006C0D002000D0272453
:108B0000983A0000E0000020EC000020E70300009D
:108B10003013002000AEFCFFDA000020F853E3A57C
:108B20009B843E40BE48008800F0AEFAF07C0028EE
:108B300079D00C990988814275D00C98E17C01802C
:108B40001222B8480199FCF719FB0822B549B6482A
:108B5000FCF714FBB349B4480A220831303057E11E
:108B60000846FDF7D9F8617B88420CD301222271B7
:108B700062794300521C6271AA4A0599CE3AD152D9
:108B800002990E754F75A74903220C390A540B99A7
:108B9000A64A8B8913868700C989A24851869C38CA
:108BA000216BC151B038C27CA37C1107090F264646
:108BB000994202D9032900D0B274F17C002912D065
:108BC00002229B49401DFCF7FDFA00280BD1012031
:108BD00098493074C8710A981638C2B272749148B4
:108BE0000199FCF7CBFA9348736D38181630326D43
:108BF00001F0CEFD7079002280008E491C3001F01A
:108C00008FFD7079002180001C3001F09BFD0AE08F
:108C1000324600210F2001F058FD207B002802D0B1
:108C2000002001F062FCE18B608C814200D2D4E52F
:108C3000814A80188142FAD8804801888800081843
:108C4000E178884200D2A5747D4A00210F2001F00E
:108C50003CFDA0786071734800260C38007800282D
:108C600012D1206CFDF71CF907467648018838467A
:108C7000FCF73EFA74487F1E0088414388B2684979
:108C80000880678300F000FA0020A073617B2279DE
:108C90008A1822E0634B0C3B195C00291BD0A57B92
:108CA000B3006D1CA5735F4D9C463C3DE9505D4B88
:108CB0004500CE3B77005D5B1833DD5385001A33EA
:108CC000584F5D5963466C3FFD50761C3B46603300
:108CD000491EF6B21954401CC0B28242DAD8A078BC
:108CE000032801D2A07BA07350490022887B4873DF
:108CF0000390401E31E000212BE04A4C8B006C3C7D
:108D0000E6581D1906956D68AE4220DDB646454E03
:108D10004C00B63E365B9700B446424E3C3EF65998
:108D20000796404E6C3EF55035464A3D67197D88A2
:108D30004A3E355334467A341C197A366568F55004
:108D4000069B76465E6066467E80079E6660491C8E
:108D5000C9B28142D1DB521CD2B28242CBDB334852
:108D600000214172039C2BE02E4B2E4ACE3B4F003C
:108D7000B63AD25BDA531D468A0062351E46AD58BC
:108D80003236B550314EB54218D01D469235AD58E9
:108D90000A2D13D1457A0626AC4675431E461A3E67
:108DA000FB18AD191B88AB8033464C33D21813889F
:108DB000EB8052882A8165466D1C4572491CC9B2F8
:108DC000A142D1D3174A0021204B9C3A8C00491C68
:108DD000C9B213510C29F9D3007C002805D01149E0
:108DE0000B7848788A78022B0ED0154A0021803201
:108DF0000F2001F06AFC0121052000224902000732
:108E0000FDF795FD0FB0F0BD074BC91C9B1F18184F
:108E1000FCF7B4F901F008FE642001F0ADF82FE58D
:108E2000C40000203C130020320D00204800002028
:108E3000E0000020A0110020983A0000CC000020A3
:108E400000D02724C8000020C6000020FFFF01003A
:108E500070470000F8B53C493A48086001F084FDCD
:108E60003A4800F0D1F83A4CE0823848801C00F0D3
:108E7000CBF820833548001D00F0C6F86083FF2042
:108E8000344D19306880E888002801D16420E880DA
:108E900031480178432901D943210170E98E0170DD
:108EA000E88F2071A88F6071A87AA070A8880090C0
:108EB00060622889FCF7E2FB284A294BFCF7D8FAC4
:108EC00000F0F6FF0022274BFCF720FAFCF71CFC11
:108ED00086B26681EF8831463846FCF709F9A081F1
:108EE00001460098FCF704F971438EB27D20C00062
:108EF00026817043FCF7C2FB1B4A1C4BFCF720FB8E
:108F0000FCF702FCE0817D2066823946C000FCF758
:108F1000EFF82082A0830120E083FCF711FFA082FC
:108F2000E28913491348FDF7B7FE13A0616A00F008
:108F30000DFEE98814A000F009FE298917A000F0B1
:108F400005FEF8BD419A000844000020004F0008CB
:108F5000BC0000202C0D0020000000206666666624
:108F60006666E63F00000840F853E3A59B843E4058
:108F7000FF7F0000B0140020B1EAC7A949443A209D
:108F80002564202E0D0A0000CDA8D1B6BCE4B8F4AB
:108F90003A202564206D732E0D0A0000B5A5B4CECD
:108FA000CDA8D1B6BBF9D5BECAFDC1BF3A20256454
:108FB000B8F62E0D0A00000070B586B01421684680
:108FC000FCF7F5F801250F4EED0300222946304647
:108FD000FDF7ADFC01200024019002946946009544
:108FE00003943046FDF7E2FB0320019002946946AA
:108FF000009503943046FDF7D9FB022000F0BCFF3A
:1090000006B070BD00040050008870477047000033
:10901000F8B5044600206A461080194D55222A7082
:10902000AA226A700322AA70661DEE702A71697105
:10903000144A49008918AC712246E81DFCF79EF8D5
:10904000002007E029186A468978128889186A463C
:109050001180401CB042F5DB611DA81CFCF7EAFC46
:1090600001466846018029190078C8716846407831
:10907000087221460931024800F042FBF8BD0000A9
:10908000F01300202C0D002010B51349CA8B8B8BD8
:109090009A4201D3D21ACA83104AC98BD2884A4352
:1090A0007D211018C90048430D490968401AFCF792
:1090B000D1FA0C4A0C4BFCF743FAFCF701FB0B49C5
:1090C000884201DD4A428018002800DA4018084929
:1090D0000968486110BD0000BC0000202C0D002074
:1090E00084000020F853E3A59B843E40FF7F0000EE
:1090F000B0140020034A1168382389B29943014310
:10910000116070470030014010B5FDF71DFC10BD27
:1091100010B59AB034216846FCF749F814210DA81F
:10912000FCF745F81C2112A8FCF741F81B48016820
:109130000324E402A143C21489180160FDF700FE74
:1091400017480169A143016106200090FF2001300A
:109150000290012003901020049002200990400406
:109160000B90000100240C900A946846FDF7E6FF7E
:109170000F200D9003200E900F9410940121119454
:109180000DA8FDF7C9FE81201290032080041890DD
:10919000149412A8FDF70EFE1AB010BD0070004026
:1091A0004010024010480168821511430160C168F7
:1091B0000E4A1140C16001680D4A1140016081688A
:1091C00049084900816001680122920491430160CD
:1091D000C168FD2212049143C1600021016106496A
:1091E0000448886070470000001002400C40FF886F
:1091F000F6FFF6FE0050000800ED00E070B50268D2
:1092000001239B07114C124D984203D0A04201D07C
:10921000A84203D17026B2434E683243984203D02D
:10922000A04201D0A84204D103231B029A43CB6879
:109230001A4380239A430B691A4302608A68C26208
:10924000096881620121416170BD00000008014090
:109250000014014010B5CB06DB0E0121046A9940D1
:109260008C430462016A9A401143016210BD30B51B
:109270008468FF252D021B021343AC430B43234399
:10928000836030BD826870239A430A4307210A43F2
:109290008260704730B5026A520852000262026A68
:1092A000456883697024A3439C080B68A40023438A
:1092B0000224A2438C68456014438361496841637A
:1092C000046230BD30B5026A10239A430262036A19
:1092D0004568826973242402A2430C682402144363
:1092E000202293438A68456012011A4384614968C9
:1092F0008163026230BD30B5026AFF2301339A43B5
:109300000262026A4568C3697024A3439C080B6823
:10931000A400234301246402A2438C684560240214
:109320001443C3614968C163046230BD30B5026A49
:1093300001231B039A430262036A4568C2697324CE
:109340002402A2430C6824021443012252039343D3
:109350008A68456012031A43C46149680164026265
:1093600030BD30B5036A046A64086400046284692D
:10937000F025AC43120122430A24A3430B4382612C
:10938000036230BD30B5036A1024A34303628469CD
:10939000036A0F252D031203AC432243A024A343E9
:1093A000090119438261016230BD000070B501F00E
:1093B0005BF80D4C0D4D606402E001F055F86064FF
:1093C000A842FAD10020E0822078002809D00128A4
:1093D00002D0022805D102E0FCF7CEFC01E0FFF745
:1093E0006FF900F033FF70BD480000203001CADE85
:1093F00010B5818CC90707D001684A6801235B0456
:109400009A43836A1A434A60818C890707D50168A9
:109410004A6801231B049A43C36A1A434A60818C39
:10942000490707D501684A6801239B049A43036BE7
:109430001A434A60818C090707D501684A680123ED
:10944000DB039A43436B1A434A60818CC90607D5F4
:109450000268916801231B039943836B1943916050
:10946000818C890607D501688A6801235B039A43CA
:10947000C36B1A438A60818C490612D503685A6807
:1094800001210905046C8A4322435A60026C8A4216
:1094900007D10268516803235B059943436C194364
:1094A0005160818C090607D501684A680123DB04F5
:1094B000806C9A4302434A6010BD0000F8B5002654
:1094C0000446C667FDF73AFA054620680068124F61
:1094D000000709D501212B460022490520460097A7
:1094E00000F054FA00280DD12068006840070BD521
:1094F00001212B46002289052046009700F046FAFC
:10950000002801D00320F8BD20206067A0676034E8
:1095100026740020F8BD0000FFFFFF01F8B5184CCD
:10952000C826E078002829D16079002826D10120BA
:109530006071144D686B002700281ED0686BC8212D
:10954000081A15E01048E168405C616988470F48D7
:109550000A21008848430E490880E068401CE0600A
:10956000E068C82800DBE760696BC820401A761EF7
:10957000E168814201D0002EE4DC6771F8BD000093
:109580003000002000000240640C0020CC000020CD
:10959000DC00002070B5224CE07800283FD1207913
:1095A00000283CD1012020711E4EF16900250906DA
:1095B000002933DA2156625791420AD1F0694006F8
:1095C0002CD5A079002829D0A5712089401C2081A4
:1095D00024E0A179002903D1A0710A2000F0D3FC76
:1095E00000202056CC2148430F4942182069121808
:1095F0001279B262401C00222061A256CC235A4349
:10960000895881420ADC25612078401C207020782E
:109610000E2800D12570A078401CA070257170BD67
:1096200030000020003801403C01002010B5806A65
:109630000022014640314A834A82FEF792F910BD6A
:1096400070B5846A606FA56F216889680026090675
:10965000002906DA212804D152200653204600F0C2
:1096600047F820688068400606D5222D04D15A208C
:109670000653204600F02CF8E06F10210843E06705
:109680002046FEF76EF970BD10B501460968806A84
:109690000968890614D400225A210A5201680A680E
:1096A000FF2301339A430A6001688A685208520016
:1096B0008A6001688A6840239A438A602021816712
:1096C000FEF7EAFA10BD10B5806AFEF7E6FA10BDA3
:1096D00001680A68FF2321339A430A6001688A6897
:1096E000520852008A60202181670021016670477C
:1096F00001680A68C0239A430A60202141677047C5
:1097000070B5164CE278002A0CD12279002A09D1D2
:109710000122E2700025C82903DC0222A256002A99
:1097200001DCE57070BD0123E356CC2253430C4AA3
:10973000D1500123E356CC2673439B180A460146B9
:10974000181DFBF71BFD6078401C607060780E28C8
:1097500000D16570A078401EA070E2E730000020C4
:109760003C010020F8B504462669A268E769324347
:109770006669102000253E432368324378491E68FD
:10978000784F3E4016431E6023685A68032636030E
:10979000B243E66832435A602368A2698B4201D023
:1097A000266A32439E680B273F02BE4316439E60E3
:1097B0006D4E23686D4AB3420CD1D2689207920F66
:1097C00006D0012A38D0022A34D0032A20D11EE044
:1097D00001201DE0664EB3420AD1D2680C26324009
:1097E00026D0042A28D0082A24D00C2A10D10EE032
:1097F0008B420DD1D66803229202164018D0012266
:109800009202B61A18D0B61A14D0964200D1082087
:10981000564A0126403A574FF6038B4236D100286C
:109820000CD002280DD0042812D008281FD11CE02B
:109830000020EDE70220EBE70420E9E7FDF722FC3A
:1098400008E01068C00601D5384605E04A4803E044
:10985000FDF738FC002873D062685100511881422E
:1098600005D81103814202D303E03046F4E7012515
:1098700066E0010E06025008002330185941FBF73C
:109880004DFC03210902411A3C4A55E0E169B1420D
:1098900032D1030000F081F909070A0D06250606FA
:1098A000062B0600E3E7FDF7EDFB1CE0FDF7FAFBF6
:1098B00019E010686168C00602D54808304A01E026
:1098C000304A48088018FBF713FC80B201462E4A44
:1098D00010399142CBD8511C01400007400F08437A
:1098E0002CE0FDF7EFFB616840004A08EAE7616899
:1098F000012248081204E5E7030000F04EF90907C9
:109900000A0D06260606062C0600B0E7FDF7BAFB90
:109910001DE0FDF7C7FB1AE010686168C00602D5BC
:109920004808C01902E014484A081018FBF7E0FB89
:1099300080B20146144A1039914298D82168C86013
:109940000020206660662846F8BDFDF7BBFB616815
:109950004A088018EAE7616848088019E6E70000CD
:1099600000480040F369FFEF00380140401002401A
:109970000044004000093D000024F400FFFC0F00FB
:1099800000127A000048E801EFFF0000FFB581B047
:1099900017460E4604460A9D09E0681C07D0FCF7EE
:1099A000CDFF0499401AA8420CD8002D0AD0206897
:1099B000C1693046884318D00020B842EDD000205D
:1099C00005B0F0BD20680168FF22A132914301601B
:1099D0002068816849084900816020206067A0678D
:1099E0000020603420740320EAE70120E5E700004E
:1099F00010B504491020096808620248FDF7B2FF5B
:109A000010BD00007415002001490D2088707047BA
:109A10003000002010B507480A22018A5143018412
:109A2000FEF7CCFCFEF7E4FDC82203490348FEF72D
:109A3000D7F810BDBC000020640C00207415002075
:109A4000F8B53D4C002321783C4A1D46082910D02A
:109A5000072945D006294ED0052950D0042951D0D8
:109A6000032952D0002954D0012956D0022958D0B8
:109A700059E0A17800264A1F04E0304FBF5DFB1873
:109A80009BB2761C9642F8DB667927799A195118B1
:109A9000E3786278C9188918C9194018C0071AD024
:109AA000012E14D0022E16D125482449C018FBF7E8
:109AB00065FB00F0B9FF642000F05EFABFF34F8F42
:109AC00021492048C860BFF34F8F00BFFDE7590808
:109AD0001046FFF79DFA2570E570A570A571F8BDD9
:109AE000A1795054491CC8B2A071A178491F88427D
:109AF000F5D1082001E0607007202070F8BDE0700B
:109B00000620FAE760710520F7E7A070E5700420F1
:109B1000F3E7552807D10120EFE7AA2803D1022057
:109B2000EBE7032803D02570E570A570F8BD03208E
:109B300020702071F8BD0000B30000208C130020BD
:109B40002C0D00200400FA0500ED00E00FB410B564
:109B500003A9044B044A029800F002F910BC08BCA7
:109B600004B01847A9A70008FC0000202021020C1F
:109B700001D010211046020A01D01046083902090E
:109B800001D01046091F820801D01046891E4208E4
:109B900001D0881E7047081A704730B47446641E9E
:109BA0002578641CAB4200D21D46635D5B00E31860
:109BB00030BC184702E008C8121F08C1002AFAD1B9
:109BC00070477047002001E001C1121F002AFBD13D
:109BD000704708B50021684601706B4601220221DA
:109BE0002C2000F081FD0221684601706B460122A5
:109BF0002C2000F079FD08BD38B504466D2069467B
:109C000008706B46012207492E2000F06DFD0649C1
:109C1000002C01D0054A00E0054A2E2000F04AFD44
:109C200038BD000006080000061800000706000006
:109C30000716000038B504466B4602220021362084
:109C400000F018FCB3212300FFF7A7FF0E0F081543
:109C50003A3A3A3A1C273A3A2F34483A00216846B1
:109C6000017040784108490014E06946087880088E
:109C70008000401C04E06946087880088000801C51
:109C800008701DE0684602780A4048320270417848
:109C9000802001436846417012E0684602780A401D
:109CA000027040784106490EF4E76946487802217F
:109CB000084303E069464878FD210840694648703A
:109CC0006B4601220021362000F00EFD012200AB80
:109CD00011463620013300F007FD38BD694608788B
:109CE000CF21084069462030CAE708B503216846FD
:109CF0004170012101706B4602220021362000F0E4
:109D0000F3FC0122D20306212D2000F0D3FC012018
:109D100000F032F90120FFF78DFF08BD08B5020AF7
:109D200069464A7008706B46022204212D2000F01B
:109D3000DBFC0320694608706B46012206212D20BA
:109D400000F0D2FC0020694608706B460122062113
:109D50002D2000F0C9FC0A212D2000F071FB08BD68
:109D6000FFB58DB00446002506E025280AD0109ADC
:109D70000F999047641C6D1C20780028F5D1284667
:109D800011B0F0BD00270121484A009700E00743C9
:109D9000641C23780846203B98401042F7D1207875
:109DA0002E2817D1042007436078641C2A280CD180
:109DB0000E98641C02C800910E900BE000990A22D4
:109DC000514330394018641C0090207801463039E6
:109DD0000929F3D920780028D1D0642808D069282F
:109DE00006D075281ED0109A0F9990476D1C5BE025
:109DF0000A200E99019001C90E91002802DA404212
:109E00002D2102E0390504D52B216A46117201216A
:109E100003E0F90704D02021F7E70BAE0B910DE02A
:109E20000021FAE70A200E99019001C90E91F7E787
:109E30000199FBF75DF93031761E31700028F7D1BA
:109E400003A8801B20300190780701D5009801E01D
:109E5000012000900199884201DD401A00E00020B5
:109E60000027009006E002A8109AC05D0F99904765
:109E70006D1C7F1C0B988742F5DB04E0109A3020A4
:109E80000F9990476D1C0099481E00900029F5DC41
:109E900005E03078109A761C0F9990476D1C019957
:109EA000481E01900029F4DC641C65E709280100C4
:109EB000F8B54A002B4B520DD6182B4A0C460546D6
:109EC000142E2BDA002E12DA284BFBF71FFA002291
:109ED0001346FBF745FD40D2002C03DA0124E407CA
:109EE00000253AE02046284337D0214C14E0214F8A
:109EF0000B46F7403B402B4331D01C4BFBF706FA97
:109F000000221346FBF72CFD27D2002C03DD012095
:109F10000005F0400419BC4300251EE0332E1EDC72
:109F200033460027143BFF43DF40384217D00F4B26
:109F3000FBF796FA00221346FBF712FD0DD2002C18
:109F40000ADD142E0CD03420811B012088404019DA
:109F5000A84200D2641C0546BD4321462846F8BDF0
:109F6000641CF9E701FCFFFF9C7500883CE4377E28
:109F70000000F03FFFFF0F007D2110B5C9004843EE
:109F800000F001F810BD002140E000BF00BF00BF9D
:109F900000BF00BF00BF00BF00BF00BF00BF00BFC9
:109FA00000BF00BF00BF00BF00BF00BF00BF00BFB9
:109FB00000BF00BF00BF00BF00BF00BF00BF00BFA9
:109FC00000BF00BF00BF00BF00BF00BF00BF00BF99
:109FD00000BF00BF00BF00BF00BF00BF00BF00BF89
:109FE00000BF00BF00BF00BF00BF00BF00BF00BF79
:109FF00000BF00BF00BF00BF00BF00BF00BF00BF69
:10A0000000BF00BF00BF00BF00BF491C8142BCD3DE
:10A0100070470000FEB50446002001900090607972
:10A02000734940000E5A61782578491E7148CFB2B5
:10A030000163042D77D0072D75D00021029121787E
:10A0400001736C49E379012292058969002B6CD078
:10A05000914381616748217A4173217A8269890736
:10A06000890B0A4382610021042000F02EFB324656
:10A0700061492E2000F01EFB3846FFF7BDFD5F4E04
:10A080000522705D810040185D49431807212B208F
:10A0900000F02AFB5B49029801220B180B212820B3
:10A0A00000F022FB705D584980000A580C212820DE
:10A0B00000F00BFBE079554980004018A179490078
:10A0C000425A0221272000F0F5FA51487E00825BB7
:10A0D0000421272000F0EEFAE079002829D0A078AA
:10A0E00004282CD028206946087220220621272027
:10A0F00000F0E0FA02AB01222621272000F0F4FA5A
:10A10000444938014018E178890042580821272045
:10A1100000F0DBFAA17A601C627A0902114313D0C5
:10A1200016E000E001E0012188E71143F6088161B3
:10A1300090E764220621272000F0BCFAE0E7102017
:10A14000694608720246D1E733490172090A417231
:10A15000417A007A0A0202432021272000F0AAFA5D
:10A160002E4F0C2123203A6800F0AFFAF0198288B4
:10A170000421232000F09EFAA07900280BD0E0797A
:10A180002749012243180021212000F0ADFA0320C5
:10A190000190012000902A07120F100102436078FD
:10A1A00000218007000B024301980005024300983C
:10A1B000400402432079C006400902436079C0068A
:10A1C00002431F2000F081FAA07861780123084340
:10A1D00002040848DB030261E179490319430A4399
:10A1E00002610021082000F070FA0020FEBD00008E
:10A1F000F4AA000800010020042800009CAA00081E
:10A20000010000201F000020A4AA0008C4AA000822
:10A21000D0AA0008D4AA000841100000BCAA000877
:10A220002100002038B50C4607498A8B00210243E3
:10A230002C2000F03FFA684604706B46012206218C
:10A240002C2000F051FA38BD0001002010B5FFF7B6
:10A25000C0FC10BD10B504460421362000F0F0F813
:10A260000121C902002C01D0084300E088430246C6
:10A270000421362000F029FA10BD000038B5402036
:10A280006946087000210E2000F0DAF8044600222A
:10A2900011460E2000F019FA6B46012200210D2014
:10A2A00000F022FA074A00210F2000F00EFA00F019
:10A2B000E7F9224600210E2000F007FA02480021AB
:10A2C000017338BDF8FF2724200100207CB5054626
:10A2D0000420694608704B4C0020607521462031EF
:10A2E000206348710873A0836063A06300F0BCF82A
:10A2F000454E206002E000F0B7F82060B042FAD18D
:10A300000020FFF797FC41480078242801D9243821
:10A3100006E00621FAF7ECFE0622101A4001084377
:10A32000020601040A4301020A43024300211E20DF
:10A3300000F0CBF96B4601220021242000F0D4F973
:10A340001E20FFF7EBFC86B2300AA0730420FFF753
:10A35000E5FC0006000E0DD002206946087101AB35
:10A36000012212212D2000F0BFF9A08B0121090349
:10A370000843A08300F078F820600620FFF7CEFCA9
:10A3800060600720FFF7CAFCA060F006C00E2075D1
:10A3900001D110202075C0B200F0E2F9E80707D023
:10A3A000FFF7A3FCA08B0121C9020843A0830AE0A8
:10A3B0000521362000F02EF81549084002460521F7
:10A3C000362000F077F90120FFF734FC002104204B
:10A3D00000F036F8A0610021262000F031F81521A8
:10A3E0008903084302460021262000F06EF900226E
:10A3F0002621362000F05EF900F036F820600020BB
:10A400007CBD0000000100203001CADE00000020F9
:10A41000FFFD000038B5094C89B280B26B460222BC
:10A4200000F028F8002806D1684640780102684606
:10A430000078081884B2204638BD0000FFFF0000F5
:10A4400038B50024E44389B280B26B46042200F0A0
:10A4500011F8002806D103216846435C2202D41873
:10A46000491EFAD5204638BD10B500210846FFF731
:10A47000E7FF10BD38B5002909D0402420436C46C1
:10A480002070C8B27F2906D8607002200AE06946B1
:10A490000870012006E0802420436C466070C809E3
:10A4A000A0700320694600F099FA38BD10B5144633
:10A4B00003460A4621461120FFF7DCFF10BD10B508
:10A4C0000346052200211520FFF7D4FF10BD10B56B
:10A4D00001210620FFF7B4FF10BD10B50346052289
:10A4E00000211720FFF7C6FF10BD38B50546002034
:10A4F0006946087000F0C4F8FF2401342246002D9C
:10A5000001D00322120200210D2000F0D3F8002D0B
:10A5100013D06B46012203210F20FFF7ABFF6846E3
:10A520000078000709D5FFF7A9FE224600210D207B
:10A5300000F0C0F80020C04338BD002038BD10B581
:10A54000024601210A2000F0C0F810BD10B50446F3
:10A5500000211A20FFF774FF000D22030005120BE3
:10A56000024300211A2000F0B0F810BD10B50246D9
:10A5700002492E2000F09EF810BD000004180000D3
:10A58000F8B505466B46012203210420FFF772FF50
:10A590000126114C3607002D0DD02A4600210C2033
:10A5A00000F088F869460878102108436946087069
:10A5B000A069304307E069460878EF210840694602
:10A5C0000870A069B0430B46A0610122032104205A
:10A5D00000F08AF8F8BD00000001002010B5024626
:10A5E0000021182000F066F810BD0000F8B50746FD
:10A5F000002568460570B807204C2E4600280ADA68
:10A600008020694608706B46012200210D2000F071
:10A610006BF801202073F8076946087821D00621DD
:10A620000843694608706B46012200210D2000F0A6
:10A630005BF803210F20FFF7EDFE8121C9000842DE
:10A6400019D04020694608706B46012200210D2078
:10A6500000F04AF80020FFF7FDFD00252673ED43CA
:10A6600009E002210843694608706B460122002177
:10A670000D2000F039F82846F8BD00002001002028
:10A680001CB56B46012203210F20FFF7F3FE68463D
:10A6900000784022C1091040C9014000814208D021
:10A6A000012069460871024601AB03210D2000F02C
:10A6B0001BF81CBD08B56B461A70120A5A7089B295
:10A6C00080B2022200F010F808BD38B500236C46B5
:10A6D000E254120A5B1C042BFADB89B280B22346D7
:10A6E000042200F001F838BD38B58024002909D0D3
:10A6F000C02528436D462870C8B27F2907D86870E6
:10A70000022009E0204369460870012004E020434C
:10A710006870C809A8700320694600F09BF938BD2D
:10A7200010B51446012312189B029A4202D9002048
:10A73000C04310BD0B46821E21460920FFF7D4FFFF
:10A74000002010BD10B5054A8905126901430A436E
:10A7500000210820FFF7B9FF002010BD00010020F4
:10A7600038B504466B4601220E212B20FFF782FEEE
:10A7700068460078E10640094001C90E0143684679
:10A7800001706B4601220E212B20FFF7ADFF38BD73
:10A7900010B5002142541C06120A22431B0A491C10
:10A7A0000429F7DB10BD000013B501231A466946E2
:10A7B0000248FDF773FA00981CBD000074150020D4
:10A7C000FCF7CAF8FEF7A4FCFDF70CFE404941482F
:10A7D000002522C005608561C5613F490562C160F1
:10A7E0000838FCF7DBF9FDF703FFFDF79FFEFDF7E7
:10A7F000B1FDFDF7E3FD052601223607D103304602
:10A80000FCF795F8FEF726FBFDF7A8FCFBF768F9C7
:10A81000FBF740F9FDF7B2FA0721B015FFF702FD8B
:10A82000FFF714FD2D4C0A21208A01224843208481
:10A8300011033046FCF77BF82648C8222849C4306B
:10A84000FDF7CEF9274F284EE07800283CD0FEF7E0
:10A850005FFCE570FBF75CFB20700F280AD9012232
:10A8600011033046FCF763F8FEF7A0FD002201213A
:10A87000090309E0012251033046FCF758F8FEF7BE
:10A8800095FD0022012149033046FCF750F8FDF701
:10A8900099FB208C002801D0401E20841348218C75
:10A8A00000780843D0D13878002801D00328CBD1D4
:10A8B0000121C9023046FCF735F80028C4D1012136
:10A8C0000846FCF75DFABFE7FDF77CFBBCE700003C
:10A8D000007C0040B0140020FFFF0000BC000020FE
:10A8E000640C00205A0000200004005036000020B4
:10A8F00010B586B01748FCF7D6F814216846FAF769
:10A9000056FC15480090032001900020029005207D
:10A9100069460007FBF74AFF69461048FBF746FF08
:10A9200069460F48FBF742FF01210846FCF728FA69
:10A93000FF2401342046FCF7FBF90A490868042289
:10A94000104308602046FCF703FAFCF709FA06B04A
:10A9500010BD0000B0140020FFFF000000040050F4
:10A96000000800500070004010B501229202184902
:10A970001848FBF72BF91648174902888A4225D058
:10A98000018004218180FF21F531C1800A210181EC
:10A9900000211E224181D24382810122C281018491
:10A9A000018241828182C182018381834323C386E4
:10A9B00002230387782343878287C2870246403277
:10A9C000118451849184C18300F02EF810BD0000E1
:10A9D0002C0D002000FC0008AA550000F0B58C46A4
:10A9E00000251026052109078E620E4C08E06746F7
:10A9F0007F5DE760A768FF07FCD0E7681F706D1CEC
:10AA00008542F4DB0020074606E0E760A568ED0715
:10AA1000FCD0E5681D54401C9042F6D38E610020A6
:10AA2000F0BD00000030014070B572B60124074D42
:10AA3000A40221462846FBF7AFF8002804D022469E
:10AA400003492846FBF74CF962B670BD00FC0008CC
:10AA50002C0D0020F0B50025102605279C463F0749
:10AA60000B46BE620C4C06E0595DE160A168C90767
:10AA7000FCD0E1686D1C8542F6DB002007E06146F2
:10AA8000095CE160A168C907FCD0E168401C904204
:10AA9000F5D3BE610020F0BD00300140000001028E
:10AAA00003040005405C0000A05C0400C06C0800CA
:10AAB000805C0400E03F1E00E07D1E0007A9022527
:10AAC00070889B880A001600010006000100020041
:10AAD00087008D002D001A3152001A339A001A3562
:10AAE0001D011A376B003B31BE003B335E013B3525
:10AAF00096023B37000099599959EB518F421E45F8
:10AB0000142E0080EB51F5283333E13A703DE13AE1
:10AB1000C235852BC2353333C235C235AE47E13A33
:10AB20005138A3305138000000000000000001023D
:10AB3000030406070809030406080C101820300057
:10AB4000000000010203040068AB000800000020C0
:10AB500000010000B49B000868AC00080001002060
:10AB6000A0190000C49B000800070400091E080586
:10AB7000400826091040085608054008261D040014
:10AB800008BE1D040008BED8BC401008010000002B
:10AB90000000C842000000000000000000000000AB
:10ABA00000000000000000000000000000000000A5
:10ABB0000100000000000000000000000000000094
:10ABC000000000008C0A00000000000000000000EF
:10ABD0000000000000000000000000000000000075
:10ABE0000000000000000000000000000000000065
:10ABF0000000000000000000000000000000000055
:10AC00000000000000000000000000000000000044
:10AC10000202140009090102008100000000000086
:10AC20000100000000000000000000000000000023
:10AC30000000000000000000000000000000000014
:10AC40000000000000000000000000000000000004
:10AC500000000000000000000000000000000000F4
:08AC60000000200000000000CC
:04000005080050C1DE
:00000001FF
